:020000020000FC
:040000000C948200DA
:1001000000EC05BFC0EDD0E000E003500DBF01E002
:1001100000400EBF0E944701002309F424D0E0E60E
:10012000F0E002E010E00E94CB16E0E0F0E000E03A
:1001300010E040E050E00E94BD16E4E0F1E00CE584
:1001400013E00E94CB16EEE3F2E000E011E044E0A1
:1001500050E00E94BD16EAE6F1E000E614E040E05F
:0A01600050E00E94BD160C94490106
:04028E0001E00895EE
:100292000E945907002319F40E947003FDCFF894BD
:0C02A2000E94A30178940E94C201FDCFCD
:10016A000A53494F32494445207665722E20332E70
:10017A00312028632932303032204D4D536F667456
:02018A000A0069
:1002AE00579800930602109307020027009304024A
:1002BE0000930502E0E6FF27F083579A089512D0C7
:1002CE00015010400C5F1E4FE02FF12F8083E0E6AF
:1002DE00FF2720E630E0082F11274081040F1F1F53
:1002EE0011500895E4E0F2E0008111810F5F1F4F7D
:1002FE0000831183089519B71D7F19BF00930A0259
:10030E0009B7026009BF089509B70D7F09BF0091B3
:10031E000A02002311F0002701C001E019B7126094
:10032E0019BF08950EEFE7DF04E010E0B9DF949AED
:10033E0001E00093080208958C9A909A07E109B99A
:10034E0008E90AB98A98929A07EB02BF05E003BF43
:10035E0009B7026009BFE6CF000F111F202F312F02
:10036E0001501040232B11F00000F8CF08955D9B33
:10037E00FECF0CB908950E94DF16A4E0B1E0C4DFF1
:10038E00002309F0CFDF00910802E2E4F2E00C94C2
:10039E006016829B9CC00EEFAEDFEA2FFB2F4181D1
:1003AE000A2F1B2F0E947B07002309F48FC0002702
:1003BE00009309029AD0E457FE4FC895002009F425
:1003CE0083C093D0E457FE4FC895EA2FFB2F0181CF
:1003DE000016E1F48AD094D00029C1F086D090D0D6
:1003EE00E02FF02D46E052E00A2F1B2F0995002337
:1003FE0069F07BD0E157FE4FC8950092080200913C
:10040E000602109107024CDF949861C00091090218
:10041E000395CECF08EC10E05DD009F44CC065D04A
:10042E00E057FE4FC89562D009F445C003E49FDF44
:10043E0007E034C040C03FC00AEF10E08DDF7DD032
:10044E0018F567D0EC5FFE4F008191DF00E610E0FB
:10045E0060D0EC5FFE4F20813327E0E6FF2740811E
:10046E00240F311F315055D028F0EC5FFE4F208104
:10047E00239503C0EC5FFE4F2081E02FF12F00810A
:10048E00020F00832FDFDBCFE0E6FF2700811DC0C8
:10049E003ED002E030DF01E46ADF04E000930802A0
:1004AE0016C000ED17E016D031F01FD0E057FE4F0A
:1004BE00C8951CD021F405E408C029D039D003E436
:1004CE0004C004EF11E048DF0EE451DF2BDFE4E05F
:1004DE000C94F01641DF2CD021D0E057FE4FC8957A
:1004EE00002D3196C8950029089518C0002D31961B
:1004FE00C895E02FF02D04E011E009950023089532
:10050E00E357FE4FC895002D3196C895089508EC17
:10051E0012C0E0910402F0910502089500910902C3
:10052E00112746E050E00E94C115E02FF12F0895EB
:10053E0001E41DDF0AEF10E00FCF009104021091CD
:10054E000502209106023091070202171307089543
:10055E000A921A922A923A920A931A932A933A93E9
:10056E004A935A936A937A93EA93FA93FFB7FA935C
:10057E008A938CB182991AC0009108020130B1F4AD
:10058E0044D050F49CDE082F08F00395E22FF32F91
:10059E001081100F10830AC0E0E6FF2700810817B4
:1005AE0011F402E001C008E000930802829B1BC018
:1005BE00009108020430B9F428D048F480DE08F027
:1005CE008395E22FF32F0081080F00830CC00EEFEE
:1005DE0092DEE0E6FF270081081711F405E001C066
:1005EE0009E0009308028991F991FFBFF991E99111
:1005FE00799169915991499139912991199109915D
:10060E003990299019900990189502E074DE95CFD3
:10061E000A93EA93FA93FFB7FA9300910A020E3FF8
:10062E0049F000910A02002329F000910A020150BC
:10063E0000930A0207EB02BFF991FFBFF991E9910E
:04064E000991189561
:1002420002006E020900D0014F026E025802110232
:0802520023026D026802640240
:04002C000C940F031E
:040034000C94AF0277
:10065200000F111F221F331F35D0015010402040C0
:100662003040452B462B472B11F00000F5CF089563
:100672002ED00E942316742E7394082F192F2A2F1E
:100682003B2FE42D24D00E942316E42D23D00E9478
:100692002316642E2A2F3B2FE42D038114814281DD
:1006A20055270E94C115402F512F66277727082F03
:1006B200192F0E942316402E512E062D0F70005620
:1006C200602E0895402F512F622F732F089543817A
:1006D200548102C04281552766277727089500EA90
:1006E20016E821E030E0B4DFAD9800E41DE023E03D
:1006F20030E0AEDFAD9A089531E040E811273323B0
:1007020039F0202F232309F0142B330F4695F7CF0E
:10071200012F08959A938A93902F042F852FECDF4F
:100722001FEF1ABB17BBF89415B3107E192B15BB1C
:10073200AF980BBB88BBAF9A000005B30F6105BB36
:1007420078940FEF0ABB0BBB07BB08BB8991999149
:1007520008959A938A9311271ABB1FEF1BBB112787
:1007620017BB1FEF18BBF89415B3107E102B15BBE7
:10077200AE980000AE9A09B386B315B31F6115BBDC
:1007820078941FEF1ABB1BBB17BB18BBB5DF182F22
:100792008991999108950E94E016A02F80E197E235
:1007A200AA2339F00197082F092B19F4AD980027D5
:1007B20005C00DE1CEDF00309CF301E0E3E00C94D4
:1007C200F1160E94DF16802FA0E1B7E2882339F0EC
:1007D20011970A2F0B2B19F4AD98002705C00DE1D4
:1007E200B8DF03FFF3CF01E0E4E00C94F0160DE173
:1007F200B0DF00FF03C0AD9801E00895AD9A002775
:10080200089525D0B0F0E42DF52D01850030042F98
:100812002CF0152F262F372F2BDF01C028D011D017
:1008220041F02ED041E209D021F03ED011F401E096
:1008320001C00027E8E00C94EC1650E00DE16ADFFD
:1008420036C005E086DF01E0A6DF002308950E949E
:10085200DB16402E512E842F952FA62FB72FE02F77
:10086200F12F29D004171507260737070895702E90
:10087200492E5A2E6B2E0FE0602200EE600E089574
:10088200462D552709E146DF41E050E009E042DF0D
:10089200472D55270DE03EDF442D552701E13ADF74
:1008A200452D50E005E136CFA2DF0023089501E097
:1008B20088DF0023089505811681278130850895F8
:1008C200C6DFB8F0E42DF52D018506FD12C0E42D3A
:1008D200F52D01850030082F2CF0192F2A2F3B2FE0
:1008E200C7DE01C0C4DFADDF21F0CADF41E3A5DF0F
:1008F20011F4002701C001E0E8E00C94EC16082F87
:10090200192F2A2F3B2F42E00C941A160E94DF1651
:10091200802F912F2AD0A0E0B1E0E02FF12F218586
:1009220026FF0EC0222733273A932A937A936A939B
:100932005A934A93402F512F082F192F54D112C086
:1009420060DF002371F00A2F1B2F1197012B01E0AA
:1009520049F0FFDEE82FF92F019311938E2F9F2F7D
:10096200F2CF0027E8E00C94F016042F152F4C81EB
:100972005D816E817F8108950E94DF16A02FB12FC5
:10098200F4DF80E091E0E02FF12F218526FD12C0F7
:1009920097DF002379F0082F192F0197012B21F0FF
:1009A2004D915D910ED0F7CF0ED021F07DDF11F485
:1009B20001E001C00027E8E00C94F016A02FB12F4F
:1009C20040CF01E0A7CE01E03FCF0E94DD16F6DF67
:1009D20009F46AC071D04CEE30DF09F465C064DFFF
:1009E20009F062C04424552401E0501608F042C0C8
:1009F2005FD0042D152DEAE5F2E00C94641600E0B8
:100A02009030A4F552C0EA2FFB2F808391832EC031
:100A1200EA2FFB2F82832AC0EA2FFB2F8383948342
:100A220025C091FF23C0EA2FFB2F018500680187B3
:100A32001DC0EA2FFB2F01850030C4F422278583D5
:100A420096832783208712C0EA2FFB2F018500306F
:100A52006CF411274581568167817085410F511FC2
:100A6200681F791F45835683678370870FEF401A8B
:100A7200500ABACFEA2FFB2F018500309CF000818B
:100A820011812227332726DE0E94F515EA2F1FDE69
:100A92000E94F515EA2F14D00EDF015010402040BD
:100AA20030400ED001E001C00027E6E00C94EE16C3
:100AB20050DE802F912F089540EA50E009E12ACEBE
:100AC20005831683278330870895BBDE11F4002740
:100AD2000895F2DF4CE050E001E11BD005E119D0AE
:100AE20005E017D009E015D00DE013D001E112DEC8
:100AF20048E050E005E10EDE40EA9FDE11F40027F7
:100B0200089561DF11F40027089501E0089550E08F
:100B120001E000DE4427552708950E94D516A02E35
:100B2200B12E442E552E662E772E88889988AE8552
:100B3200BF85CC2404E0D02EC8DF002309F449C0CD
:100B420048EA50E03EDF472D562D3BDF452D542D20
:100B5200DFDF37DF40E051E034DF3FD0D1F1002763
:100B620030DE0023B1F1A0DEA1F52C2D3D2D0FEFDB
:100B7200C00ED01E232B01E011F19ADF0A2F0B2B9E
:100B820011F011970BC0082D092941F00FEF800ECB
:100B9200901EEA2DFB2D8193AE2EBF2E0A2F0B2B1A
:100BA20011F01197E2CF082D0929F9F20FEF800E0B
:100BB200901EEA2DFB2D9193AE2EBF2ED6CF01DED5
:100BC200002329F001E0C5DD72DEE1F702C001E099
:100BD20001C00027E2E10C94E6164427552701E004
:100BE20099DD002731CE0E94DB16602E712E4C84D7
:100BF2005D8488859985AA85BB85E42FF52F0185BB
:100C020006FF58C058DE80179107A207B30708F005
:100C120051C001E0401602E0500608F04BC0042D1E
:100C22000529B9F1082F0370112722273327033032
:100C320010402040304069F562DE802F912FA22FB4
:100C4200B32F00E012E0041915091A930A93042D38
:100C5200152D1A5F1A930A93482F592F622F732F5B
:100C62002FD009F427C08F5F9F4FAF4FBF4F5A92CB
:100C72004A92002711271A930A93482F592F6A2F55
:100C82007B2F64187508600E02E0701E19D0A1F463
:100C920011C000E012E01A930A93082F0370102F7C
:100CA2000027110F040D151D1A930A9328DE0ADD81
:100CB20007D011F4002701C001E0EEE00C94EC161D
:100CC200062D172D2ADF002308959A938A931A93EB
:100CD2000A93842FFADE002369F04BE151E018DF1A
:100CE20070DE482F50E014DF13DF6BDE76DF11F089
:100CF200DBDD11F0002701C001E022968991999174
:100D0200089542E0E2CF43E0E0CF0E94DF1656DED4
:100D120069F1D2DE41EA91DD49F1C6DD39F5882774
:100D2200992701E09130B0F414DD282F392F20509B
:100D3200304021F02153304021F00AC0103044F0FD
:100D420015C011FF13C0EA2FFB2F01850068018730
:100D52000196E7CFEA2FFB2F01850064018700E8A7
:100D620011E327E130E0ACDE01E001C00027E4E05E
:100D72000C94F0160E94DB16402E512E642E752E16
:100D8200A4DE002319F143E0C2DE1BDE42E1BFDE36
:100D9200BFDEBEDE16DE17DEC9F089DDB9F084DD06
:100DA200A9F4AA27BB27EA2FFB2F399701E078F491
:100DB2007FDE0A2F1B2F0650104031F4E42DF52D53
:100DC2008083E62DF72D90831196EDCF0027E8E082
:100DD2000C94EC162297E02FF12F018506FF12C02A
:100DE2004C2F5D2F4F5F5F4F0C2F1D2FC3DF002352
:100DF20049F00881E4E7F2E00C94601601E003C0D8
:100E0200002701C002E0229608959A938A93802FC8
:100E1200912F0027E82FF12F0083018302830383A0
:100E2200048305830683078300870187082F6DDF0C
:100E32000023082F192F41F066DF082F192FCADF70
:100E42000130D9F702E006C0C0DD002311F001E055
:100E520001C000278991999108952EDE4EE050E05D
:100E62000AE158DC0AE010E020E030E0F1DB4AE081
:100E720050E00AE14FDC00E211EA27E030E0E8DB73
:100E8200002789CC9A938A93802F912F0FEF0ABB68
:100E92000BBB07BB08BB04BB0FE105BBAE9AAF9A05
:100EA200AD98DBDF082F192FB0DF89919991089552
:10025A0000000137050005010405020905030D0523
:10026A002B12050B1A05012505FB00010307FF06E2
:10027A00020307020307240307010307110107C545
:03028A000307FB6C
:100EB2008D988E988F98959A969A979A00B300304B
:100EC2008B9A14F0939801C0939AE1E6FF27F0837E
:100ED2000E946414002321F48B9A939A00270895A8
:100EE20000B300300CF08B9A939A01E0E1E6FF2701
:100EF20000830895E02FF12F2081213711F4859B83
:100F020007C0E02FF12F2081223701F5859B1EC0FB
:100F12004131C1F04231B1F04631A1F0433191F09B
:100F2200443181F0453171F0473161F0483151F07F
:100F3200493141F04A3131F04B3121F04C3111F05D
:100F42004D3111F401E0089500270895E02FF12FAB
:100F52002081213318F02081293310F000270895D1
:100F620020B320303CF4E02FF12F2081213311F403
:100F72000027089586990EC0E02FF12F208121339A
:100F820011F422E306C0E02FF12F2081223311F465
:100F920021E32083E02FF12F008100530E943312BE
:100FA200012B11F001E0089500270895E02FF12FA1
:100FB2002081205320930B022381028100930C0293
:100FC20020930D0200910B020E94331220910C0219
:100FD20030910D020217130708950CD00CE010E0B7
:100FE200E42FF52F0083118300910B020E9433122C
:100FF200012B0895E02FF12F0081005300930B0283
:1010020008951DD031F0D2DF20F0022F132F032BD1
:1010120011F4002711C0E22FF12F319738F0E22F9F
:10102200F12F349718F400E810E001C015D0E82F32
:10103200F92F0083118301E08991999108959A9380
:101042008A93842F952FE1E6FF272081222308959A
:101052009A938A93802F912F00910B020C94211264
:1010620002D00C9443131A930A9340910C025091AC
:101072000D0200910B020895E2DF31F097DF20F0BC
:10108200022F132F032B11F4002711C0E22FF12F8F
:10109200319738F0E22FF12F349718F400E810E07E
:1010A20001C0DADFE82FF92F0083118301E0899173
:1010B20099910895D8DF0C94C8129CDF04E00FD0F8
:1010C2000AD0012B11F400270895E1E6FF270081E1
:1010D20008958E2F9F2F00910B020C94331210E073
:1010E200E42FF52F008311830895B2DF0030114001
:1010F20011F400E301C000E1E82FF92F01930FEF93
:10110200019300EE01930027008301E089919991F8
:10111200089563DFD1F600270895D7CF9A938A9373
:10112200802F01E0E82FF12F019300E10193D1DF3D
:10113200E82FF92F1193CDDFE82FF92F0193002724
:1011420001938E2F9F2F88DF0030114041F40CE075
:10115200E82FF92F019301E00193002707C008E06F
:10116200E82FF92F01930027019300E8019300E48F
:10117200019309E4019304E4019305E4C5CF2DDF53
:1011820009F0A3CF00270895A0CF9A938A93E02F66
:10119200F12F8281982F0381802F9DDF0817190775
:1011A20011F0002701C001E08991999108959A9365
:1011B2008A93842F952F1EDF0E942112E82FF92F88
:1011C2000083118300811181012B11F4002703C0D8
:1011D200E1E6FF27008189919991089539DF025054
:1011E20010402FEFE82FF92F21932193202F312F39
:1011F20001501040232B09F488CF2227F6CF85CF48
:101202001A930A930027E42FF52F00830183229675
:1012120008951A930A93002722960895E02FF12F3A
:10122200028100930B020FE05ADF00910B020C9433
:101232001912402F512F00910B020C943D11EECF49
:10124200402F512F00910B020C9468111A930A93AC
:101252000FE045DFE1E6FF270081229608950C9416
:101262000D11F4CF0C94291121E030E0E42FF52F79
:1012720020833183E02FF12F02810C94FB112FEF99
:10128200E02FF12F208321CF1A930A9301E0E1CFBF
:101292002FEFE02FF12F20830C9447121A930A9319
:1012A2000AE0D7CF0E94B01201E008951A930A9380
:1012B20004E0CFCF0E94B61201E008951A930A9378
:1012C2000FE0C7CF0C94B510F9CF0C94C810F6CF2D
:1012D2000C94D810F3CF0E94E51001E00895EECFF0
:1012E2009A938A93802F912F0E94CB13002339F077
:1012F200082F192F0E94E5100E94091106CF0FE056
:1013020010E01A930A9344275527082F192F0E9499
:041312003617FBCEC1
:10018C00535E08067608500208033108570208032C
:10019C003108523D08065B084E8A08068F084FC08E
:1001AC000803C60821D80806EF083F0109060A090A
:1001BC00110F09061A091220090321091327090630
:1001CC003009143209063309164509064909153553
:1001DC0009064009174F09065309185709065B0908
:1001EC00195F090663091A65090666091B68090384
:1001FC0069091C6B09066C091D7009067109000060
:04020C0000010000ED
:101316000E94DF16802F912FA22FB32FE0E0F1E07D
:1013260061D069D089F0BA93AA939A938A936CD0C4
:101336000E948704002311F4002707C0E0E0F1E0D3
:1013460080839183A283B38301E0E4E00C94F016DA
:101356000E94DF16802F912FA42FB52F5AC0222767
:10136600332701505CD05FD0802F912FA22FB32F4F
:10137600082D5FD0E25FFB4F00811181228133810E
:10138600800F911FA21FB31F0895041B150B260B78
:10139600370B40914A045527662777270E94231664
:1013A600802F912FA22FB32F8E5F9F4FAF4FBF4F2E
:1013B6000895802F912FA22FB32F823000E01007BF
:1013C600200730070895802F912FA22FB32F0F3FAC
:1013D6001F4F08950E94DB16602E712E442E552E47
:1013E600E5E5F4E0008111812281338108958F5F64
:1013F6009F4FAF4FBF4F80179107A207B3070895BE
:101406003A932A931A930A934BE454E00EE012E0BF
:10141600089541EC5DE09CD20023089502501040EF
:10142600204030400895442D552D662777270C948B
:101436002316112747E050E00E94C115E02FF12F37
:1014460008955A934A93DCDF0C94F405D9DF0C9483
:10145600BD040E94DF16802F012F122F232F332762
:1014660031D019F40027112705C0E82FFF2734D003
:101476000081118122273327E4E00C94F016082F0F
:10148600CDDF40914A045527662777270E94F51538
:1014960035D03BC0E8E3F4E03DC0E8E3F4E0058482
:1014A60016842784308881859285A385B48508169D
:1014B60019062A063B06089521D0401751076207F0
:1014C60073070895E8E3F4E04181528163817481F2
:1014D6001CD01EDF00230895EE0FFF1FE25FFD4FB5
:1014E6000895E8E3F4E00584168427843088E5E56A
:1014F600F4E000821182228233820895E8E3F4E068
:1015060045815681678170850895040F151F261F32
:10151600371F0895018512852385348508950E9415
:10152600DF16802F47E00E941A16CCDF29F4002729
:1015360011272227332708C0E82FEF77FF27EE0F62
:10154600FF1FCADF4FDF3F70E4E00C94F0160E94E5
:10155600DB16602E712EE02FF12F44DFADDF28F46D
:10156600E62DF72D3FDF11DF01C050D0442455246E
:1015760000913804045039F0025029F00650E9F081
:101586000357B9F139C0082F192F2A2F3B2F61DFD6
:10159600402F412B422B432B79F14FEF441A540A2B
:1015A6000F3F140740E02407340711F020DF21F530
:1015B6000ADF2040304039F719C0082F192F2A2F8B
:1015C6003B2FADDF402F412B422B432BA9F04FEF92
:1015D600441A540A0F3F140724074FE0340711F04A
:1015E60006DF51F4F0DE2F4F3F4039F7042D152D5D
:1015F6000AC001E010E007C0E62DF72D0681006263
:10160600068300271127E8E00C94EC1682E090E0B0
:10161600A0E0B0E0089511D0065F1F4F0E94641548
:101626000051FDDE442D552D662777270C94231691
:10163600042D152D262D372D089500915B0410914C
:101646005C0408950E94DF16802F912FA42FB52FDA
:10165600C7DE56DF3CD090F500915904112745E0CE
:101666000E94D115025F1D4F00935E0410935F0424
:10167600009159040031E0F4B5DE32D011F40027B0
:101686001EC000915904039500935904082F192F81
:10169600EA2FFB2F0995002311F001E010C0E5E5C4
:1016A600F4E001851285005E1F4F01871287E0CFA7
:1016B60000270093590496DE05D0CACF02E0E4E085
:1016C6000C94F0160F5F1F4F2F4F3F4F11C004179A
:1016D6001507260737070895082F192F2A2F3B2F9E
:1016E600F8CE018712872387348707C0E5E5F4E043
:1016F60000831183228333830895058716872787FE
:10170600308B08959FDF002339F00A9519F00A956A
:1017160019F002C001E00895002708950E94DF161F
:10172600A02FB12F842F952FB5DEE0DF0DD01BD073
:1017360018D0002700935904482F592F0A2F1B2F22
:10174600E1DFE4E00C94F01600914A041127409181
:10175600490455270E94C115212F210F220B322F34
:101766000895D3DE05C04081518162817381089559
:10177600058316832783308708952CDE9DDE10F4BB
:1017860004DE01C043DF3FD039F00A9519F00A950F
:1017960029F004C001E011C000270FC0082F192F3F
:1017A6002A2F3B2F56DE05DE10F069DE01C072DE01
:1017B60007D000E0A007B00731F7E8E00C94EC167C
:1017C60095DF00914A04112722273327CCDF9DDEBF
:1017D600CFDF8F3F0FEF90070895442D552D0E94C0
:1017E600DF1541505040042F152F462D572D0C94D0
:1017F600C115442D552D0E94DF15452B082F192F95
:101806002A2F3B2F0895442D552D062D172D1ADF0F
:101816000023089504D0B1DFE4E00C94F0160E9492
:10182600DF165FDE00904A041124222433248081CF
:101836009181A281B381080E191E2A1E3B1E0582C4
:101846001682278230862227209359040895C2DD06
:1018560033DE10F49ADD01C0D9DED5DFB9F00A9582
:1018660019F00A9521F003C001E011C00FC0082F3E
:10187600192F2A2F3B2F53DE9CDD10F000DE01C00E
:1018860009DE9EDFA0070FE0B00739F70027E8E082
:101896000C94EC16C4DFDBDFE4E00C94F0160E9437
:1018A600DD16802F912F442E552E9ADD19DFF1F08B
:1018B6000091590410915A04025F1D4F39D0B1F0BE
:1018C6003FD00E94391511272091590430915A04AE
:1018D600020F131F125098F0422F532F81DDB1DDF6
:1018E600002321F00EE012E023D011F4002710C0EF
:1018F60012D0132F1170158375DDE4DE01C00BD0F5
:10190600082F192FE42DF52D0995002371F201E01A
:10191600E6E00C94EE1691DE0E9439151127E5E5F6
:10192600F4E024813581200F311F24833583089507
:1019360000935B0410935C040E94391500230895FC
:101946007CCECFDD22272093590420935A04A7CFBB
:101956000E94DF1620913804245039F0225029F0D5
:10196600265049F0235749F00AC097DD11F4D6DE18
:1019760007C050DF05C08EDF03C0E3DF01C00027CC
:10198600E4E00C94F0160E94DF16209138042450EF
:1019960039F0225029F0265049F0235749F00AC061
:1019A6007CDD11F4AFDE07C0E8DE05C050DF03C002
:1019B60076DF01C00027E4E00C94F0160E94D716EB
:1019C600802F912F842E952EAC84BD84E02FF12F8D
:1019D600B0A170D040E250E0082D192D0E943617B4
:1019E60003E069D040E250E00A2D1B2D0E94361715
:1019F600BB2309F445C0BF3008F042C0E82FF92FD9
:101A060001A10230E8F1482E592E01E2400E00E015
:101A1600501E6B2EAA274BE337D031F057D020F457
:101A2600B02F082F0F5DB01BBD3050F54EE22CD005
:101A360069F04CD058F4602E282F2F5D621A0F5F84
:101A46001F4F402E512EAB2FA619AA9509E06016FE
:101A5600B8F4A430A8F477247A926A928196482F33
:101A6600592F082D192D0E941F17BB27BA93AA9329
:101A7600442D552D0A2D1B2D0E941F1701E001C074
:101A86000027EEE00C94E81650E0082F192F0F5DA2
:101A96001F4F0E944717202F212B0895402F512FAB
:101AA600622F732F062D172D24D0402E512E012B79
:101AB60008951AD008E010E01A930A9308950E9438
:101AC6001F17082D192D2A2D3B2D0895282F392F44
:101AD6002F5D3F4F402F512F421B530B4B1750404A
:101AE60008950F5F1F4F28CF0087118722873387FE
:101AF60008953FD0042F152F262F372FF1DD49F1FA
:101B06002EE032E000910E0210910F0206391240CB
:101B160029F0E82FF92F068500610687E22FF32FBB
:101B2600048115810030114029F4E82FF92F06852C
:101B360000640BC0E22FF32F04811581003810409A
:101B460029F0E82FF92F06850061068749DCC8DDF4
:101B560019F4002711270AC0E82FF92F068506FF7A
:101B660003C000E011E002C000E810E089919991FD
:101B760008959A938A93802F912F08950E94D716DD
:101B86002397602E712E0FE096DF44275527062DEA
:101B9600172D0E943617009138040F3709F062C0DE
:101BA600CFDEF6D0012B022B032B09F4ACC0C8DE26
:101BB60098DF09F0A8C00C2F1D2F1A930A93462D03
:101BC600572DBEDEFBDE002309F49DC0E0915B04C9
:101BD600F0915C04018D01FD96C0E62DF72D06857A
:101BE6000460068703E067DF4DE152E00C2F1D2FEE
:101BF6000E5FDED069F4A4DECBD001301240204067
:101C0600304008F080C008E0E62DF72DBCD024C097
:101C160003E051DF40E152E00C2F1D2F0E5FC8D0CC
:101C260009F071C08DDE0E5F1F4F0E94641536DF0E
:101C360009F469C0F0DC452B462B472B41F080DECA
:101C4600A7D0013011402040304008F05CC0E3DCF2
:101C5600E62DF72D0487158773DE9ED0E62DF72D2A
:101C660043DF8CC0AAD0828C938C04891589A02E60
:101C7600B12E0081053E09F446C00081002309F417
:101C860042C003850E7DF9F5048D158D268D378DA1
:101C9600012B022B032B09F436C003E00CDF4DE1C8
:101CA60052E081D0C9F489D0048D158D268D378DEB
:101CB600013012402040304030F508E0E62DF72D87
:101CC6000687002711270487058702E080169106FC
:101CD600A106B106F0F546C003E0EDDE40E152E0B4
:101CE60062D089F46AD0038500FF05C0E62DF72D82
:101CF60006850460068766D018F0E3DEC1DB01C006
:101D0600C9DBCCDE11F400273AC057D0848D958DFF
:101D1600A68DB78D082F192F2A2F3B2F81DC452B37
:101D2600462B472B39F0813001E0900700E0A007F1
:101D3600B00728F580519040A040B040082F192FD9
:101D46002A2F3B2F70DBE62DF72D048715873AD017
:101D560048F00EEF800E0FEF901EA01EB01EB1DEF3
:101D660090DB01C097DBE62DF72DA3DE40915E04E4
:101D760050915F04062D172D0E941F1701E0239630
:101D8600ECE00C94E816068700270487058708957B
:101D9600065F1F4F0C9464150E5F1F4F0E9464155B
:101DA60042E00C94111600915E0410915F04085FE6
:101DB6001F4F0E949F14012B0895E0915E04F0913D
:101DC6005F04089502E0801600E09006A006B006C3
:101DD6000895BEDA59F06EDE4A2F5B2F082F192FB1
:101DE600E8DF11F401E003C005D0A9F70027E4E01D
:101DF6000C94F01641EC5DE0082F192FC4DD00238A
:101E06000895A6DA69F056DE4A2F5B2F082F192FA0
:101E16000E94FB16012B11F401E003C0EBDF99F7DA
:101E26000027E4E00C94F01693DA61F0E82FF92F1E
:101E36000DD0EA2FFB2F97DC4ADC11F401E003C03A
:101E4600D9DFA1F70027E4E00C94F0160085118590
:101E56002285338508959A938A932F970027112711
:101E6600222733273DDC09F472C02EE032E0EEE093
:101E7600F2E0E250FE4F0081118105351A4A09F061
:101E860066C022543E4FE22FF32F0481009338049C
:101E9600DDDF26DC09F45BC08EE092E000913804B9
:101EA600045029F0025019F0065029F150C054D0C0
:101EB600438554856BD041875287638774874587EE
:101EC60056876787708BE82FF92F0681178144E0C4
:101ED6000E94D815177F40914A0455270E94DF15A6
:101EE6000093490431DCE8E3F4E0418552856385DB
:101EF600748537DC2AC030D0418D528D47D045835A
:101F060056836783708701E000934904E82FF92F11
:101F160001A112A123A134A1023081DA30F001A17E
:101F260012A123A134A1ACDA01C0B4DADADBF2DA09
:101F3600088719872A873B8700270C870D8746D095
:101F4600202F212B11F00093490401E001C0002746
:101F56002F968991999108950B96E82FF92F41892B
:101F66005289638974890381148122273327400F9C
:101F7600511F621F721FE8E3F4E0418352836383BB
:101F86007483E82FF92F0581112708950E94C11542
:101F9600228120934A044189528963897489038086
:101FA6001480400D511D631F731F2227400F511FC0
:101FB600631F721FE8E3F4E008950C2F1D2F085FDE
:101FC6001F4F1A930A9341E252E008950C2F1D2FDA
:101FD600085F1F4FBCCA9A938A9300E410E020E082
:101FE60030E07EDB51F18EE092E00EE012E00E94DE
:101FF6003915013011F505E05EDD48E352E00EE0EB
:1020060012E00F5FD5DEC9F40FE7009338040EE047
:1020160012E004561F4FC0DEE8E3F4E062DB805BAB
:102026009F4F082F192F0E94641542E00E94111637
:10203600EBE4F4E09DDB01E001C000278991999172
:1020460008959A938A93992781E0863038F4082F69
:102056000AD00CD00CF493958395F7CF092F89916C
:1020660099910895082DE5C9402F512FEC5EFB4F3D
:102076000081003008959A938A93239763D0009144
:1020860038040F3721F55CDC83DE00301840204031
:102096003040A9F555DC25DD91F50C2F1D2F1A933F
:1020A6000A93482F592F4CDC89DC002341F1E0913B
:1020B6005B04F0915C04018D01FF21C0E82FF92F2C
:1020C6000685046060DE3CDC67DE43D036C075DE24
:1020D600028D138D44895589242F352F4081453E25
:1020E60071F04081442359F0438544FF08C0448D74
:1020F600558D668D778D452B462B472B11F0002786
:102106001DC044275527E82FF92F448745870230FD
:1021160014072407340728F081D940914A04B4D91A
:1021260001C0B8D9E82FF92FC4DC40915E04509164
:102136005F04082F192F0E941F1701E0239689912B
:1021460099910895802F912F0FE010E01A930A932A
:1021560003C0E82FF92FC8CC44275527082F192F7D
:102166000C94361706DD4EE350E1F2DB002331F026
:10217600E82FF92F06850260068703C00FE09BDC77
:10218600EBDF01E0899199910895F3DC4EE350E18C
:10219600FADB002331F0E82FF92F06850260068767
:1021A600F0CF0FE088DCD8DFECCFE02FF12F2685CB
:1021B60021FF06C04BDEE8E3F4E09FDA01E0089574
:1021C600002708959A938A93BDDFE8E3F4E0058536
:1021D600168527853089418552856385748577DA2A
:1021E60069DC19F446E252E002C04FE252E0082FE1
:1021F600192F0E94D114E8E3F4E00585168527859A
:102206003089A7DF068502600687BBCF05E414E0A8
:102216000C949F15AEDCFDD821F211D069F04ADC92
:1022260044E152E0082F192FC4DD31F0E82FF92FD1
:10223600068500680687A5CFDDDD79F7B2CF082FC2
:10224600192F085F1F4F83D9012B089592DCD2DD29
:1022560009F4A7CFF4DFD9F32DDC44E152E0082FCF
:10226600192FA7DDA1F3E82FF92F06850068068749
:1022760088CF97CF0E94DF16802FA42FB52F0FE0AF
:102286001ADC442755270A2F1B2F0E94361788234E
:10229600C1F08630B0F400911404083091F4082F90
:1022A600E2DEE2DE64F4425F5B4F0A2F1B2FBCDDE9
:1022B600002329F0EA2FFB2F06850068068701E038
:1022C60001C00027E4E00C94F0160E94DA162F975E
:1022D600802E442E552E002309F47BC006E080167E
:1022E60008F077C000911404083009F072C0485F06
:1022F6005F4F0C2F1D2F98DD002309F46AC0E5E51A
:10230600F4E080819181A281B38160DE012B09F422
:1023160060C0009138040F3709F459C0DDD909F4BB
:1023260058C0E42DF52D068548DD02FF03C0038560
:10233600016002C003850E7F0387082F192F53D033
:1023460009F447C0082D4AD0202F312F025F1B4FBA
:10235600EC2FFD2F389647E050E00E94B016E22F92
:10236600F32FEC5EFB4F008100680083E42DF52D12
:1023760006852C5E3B4FE22FF32F02FF03C0008140
:10238600046002C000810B7F0083A1E0A630F8F450
:102396000A2F24D0802F912F825F9B4FE82FF92F91
:1023A60040805180628073805DDEE25FFB4F1AD809
:1023B600401651066206730641F4A81531F0082F3F
:1023C600192F47E050E00E94B016A395DFCF01E039
:1023D60001C000272F96E9E00C94EB16112747E081
:1023E60050E00C94C1152A2F3B2F30D800230895B6
:1023F6009A938A93202F0023A9F0263098F400910F
:102406001404083079F407E056DB5527022F47E01D
:102416000E94C115025F1B4F40E050E00E94361734
:1024260001E001C00027899199910895002321F0C8
:10243600063010F401E0089500270895002369F09E
:10244600063058F410DE12DE44F406FF03C000E046
:1024560011E0089500E810E0089500271127089577
:10246600002379F0063068F4FEDDEC5EFB4F208138
:1024760020303CF40E5E1B4FE02FF12F00811181BE
:1024860008950027112708950E94DB162F970091C3
:1024960038040F3709F455C0D4DD11274DE050E05C
:1024A6000E94C115802F912F44E152E00C2F1D2F61
:1024B60090DC002309F445C0AA277FDC848F958F22
:1024C600A68FA78F0E94F30990DFD9F1488459841B
:1024D6006A847B8488279927A1E0A63080F50A2F95
:1024E600C2DDC2DD54F5425F5B4F0C2F1D2F9CDC15
:1024F600002319F19DD8F4D821F104E427D00A2F3E
:10250600005D24D00DE322D0D5DA4C2F5D2F4E5F2F
:102516005F4F082F192F025F1D4F0E941F17089645
:102526000DE014D00AE012D00027E82FF92FE25F61
:10253600FD4F00837DD859DF21F0A395CECF01E072
:1025460001C000272F96E8E00C94EC16E82FF92F2F
:102556000196E25FFD4F00830895EBE4F4E04AE064
:1025660050E00C94B01605DB00913804E82FF12FEB
:10257600008300914A04018364DDE82FF92F02836A
:1025860001E303838991999108950E94D516802EBF
:10259600A42EB52ECE84DF84002309F464C006E0A1
:1025A600801608F060C05EDDEC5EFB4F80818030F7
:1025B6000CF059C057DDEE5EFB4F008111810A1504
:1025C6001B0508F450C00A2D0B2909F44CC086FFE0
:1025D60004C0662401E0702E03C000E8602E772454
:1025E60046D00A2D1B2D0E94B2090A2D1B2D01D99A
:1025F60071F076D8C1F10A2D1B2DEFD8005F1F4F61
:102606007A926A92025F1D4F402F512F26C068D8DA
:1026160051F100E112E006191709262D372D205138
:1026260030403A932A93025F1D4F402F512F0C2DB5
:102636001D2D0E941F178F5F9F4FAF4FBF4F4CD866
:1026460091F0062D172D0051104020E130E03A930D
:102656002A934EE052E0C00ED11E0C2D1D2D0E9475
:102666001F1701E001C00027E0E10C94E61600E028
:1026760012E0462D572D0E94DF15402E512E08954B
:102686000E94D316802EC42ED52EE888F988009194
:1026960038040F3709F471C0882009F46EC006E0CB
:1026A600801608F06AC0DEDCEC5EFB4F808180306D
:1026B6000CF063C082FD61C0D5DCEE5EFB4F00818D
:1026C60011810C151D0508F458C00C2D0D2909F4AF
:1026D60054C086FF04C0662401E0702E03C000E8E3
:1026E600602E7724C4DF0C2D1D2D0E94B209882E82
:1026F600992EAA2EBB2E0C2D1D2D7BD899F00E944B
:10270600730BD9F10C2D1D2D68D8802F912F409673
:102716007A926A9236D00E941F17082D192D63DE11
:1027260061F129C00E94730B41F180E192E08619A4
:102736009709062D172D005110401A930A9321D0A0
:10274600BED953DED1F00FEF801A900AA00AB00A64
:10275600862D972D80519040B4D90E94730B69F055
:1027660000E1A9D9E80EF91E4E2D5F2D0EE012E00C
:10277600A6D93BDE11F001E001C00027E2E10C948E
:10278600E4164E2D5F2D825F9D4F082F192F089559
:102796000E94DE162A97A02FB12F44E152E019DBE2
:1027A600002309F47CC0EA2FFB2F04851585012B35
:1027B60009F075C00AE27FD97ED00EE014E074D02D
:1027C600EEE0F4E00E94F5090E94730B09F467C07D
:1027D600F4DB0EE012E00E94F714802F912F012BFC
:1027E60009F45DC0E82FF92F0081043409F044C0D4
:1027F60002810D3309F040C0418000ED400EE1F149
:1028060006E04016C8F5082F192F0D5F1F4F0E94CE
:1028160054170930104080F54DD940E250E00C2F96
:102826001D2F0E5F1F4F0E943617082F192F0D5FA1
:102836001F4F0E9454171A930A930396482F592F35
:102846000C2F1D2F0E5F1F4F0E941F174C2F5D2F41
:102856000A2F1B2FD6DA002379F00A2F1B2FB8DB9D
:10286600012B29F0EA2FFB2F068500680687042D29
:10287600B5DD025F1B4F18D0EEE0F4E00E94F509CB
:102886000E94730B61F099DB002711270E94F71451
:10289600802F912F012B09F0A5CF01E001C0002761
:1028A6002A96E5E00C94EF16EA2FFB2F389647E0C0
:1028B60050E00C94B016442755270EE014E00C9413
:1028C60036172F9703E1F7D84427552708E314E076
:1028D6000E9436170AE2EFD8EEDF0BE414E00E94FE
:1028E6004307002331F10A9519F00A9529F021C012
:1028F600B2DA002321F41DC06EDB0023D1F005E41B
:1029060014E00E946B15002329F00C2F1D2F40DFC9
:10291600002369F401E414E00E949F150E944D0A09
:102926000E94800B0C2F1D2F33DF002311F001E0D6
:0829360001C000272F9608954F
:04023E00FFFFFFFFC0
:100210004154520053494F32494445200043464718
:100220000020090D0A00433A28524F4F5429002854
:0E0230005355424449522900434430303100B6
:10293E0028813981622F732F21503040672BD9F0B7
:10294E00E02FF12F6081E42FF52FC895601571F0FF
:10295E00E02FF12F0081E42FF52FC895001618F403
:10296E0001E010E00AC00FEF1FEF07C00F5F1F4F0F
:10297E004F5F5F4FDFCF002711272296089505D0B6
:10298E000F5F1F4F008311830895E82FF92F0081E9
:10299E00118108959A938A938A819B81282F392FCA
:1029AE000197232B59F0E42FF52F4F5F5F4FC895FA
:1029BE00E02FF12F01920E2F1F2FF0CF89919991B9
:1029CE0022960895E02FF12FC895002031F0C8957A
:1029DE00041629F00F5F1F4FF5CF0027112708951A
:1029EE000E94DD16442E552E8E819F81202F212B85
:1029FE0021F0E82FF92F00831183C7DF012B41F05F
:102A0E002BD021F020D011F0BADFFACF25D019F457
:102A1E000027112715C0E82FF92FA081B1811CD0F6
:102A2E0069F011D011F4ABDFFACF0027E82FF92FA0
:102A3E0020813181E22FF32F0083A1DF0A2F1B2F7C
:102A4E00E8E00C94EE16A1DFE02FF12F4081042D6B
:102A5E00152DB8DF012B089598DFE02FF12F00819F
:042A6E0000230895A4
:102A7200E02FF12F00810895E02FF12F008111271F
:102A82000895E02FF12F008111810895E02FF12F99
:102A920020810181122F0895F4CFF3CF402F512FBF
:102AA200E02FF12F0081302F22271127E42FF52F5D
:102AB2000180322E202D33290280312E102D332910
:102AC2004381042F0895E02FF12F0081118122818B
:042AD20033810895AF
:102AD600E02FF12FE199FECF19D0E09A0DB30A3A13
:102AE60091F4E199FECF05E61BD0E199FECF06E60B
:102AF60017D0E199FECF07E613D0E199FECF08E69D
:102B06000FD001E0089500270895F89404E610E038
:102B16001FBB0EBB089510E01FBB0EBB019107C083
:102B260010E01FBB0EBBE09A0DB3019308950DBBD9
:102B3600E29AE19A78940895E02FF12FE199FECF79
:102B4600E4DF0FEFF4DFE199FECFF89405E6E3DF6B
:102B5600E199FECFF89406E6DEDFE199FECFF89420
:102B660007E6D9DFE199FECFF89408E6D4DFE199CC
:0C2B7600FECFCBDF0AEADBDF01E00895B0
:102B8200002411240030010741F01695079510F436
:102B9200040E151E440F551FF5CF002D112D08955B
:0E2BA2004A9522F0000F111F0C94D1150895D2
:0E2BB0004A9522F0169507950C94D8150895B5
:102BBE0000241124E0E1EA9552F0001F111F001CC1
:102BCE00111C04161506B8F3041A150AF4CF001FCB
:0C2BDE00111F402D512D009510950895F9
:102BEA000024112422243324E02FE12BE22BE32BAF
:102BFA0071F0369527951795079520F4040E151E42
:102C0A00261E371E440F551F661F771FEDCF002D56
:082C1A00112D222D332D089528
:102C22004A9532F0000F111F221F331F0C94111608
:022C3200089503
:102C34004A9532F036952795179507950C941A16F0
:022C44000895F1
:102C46000024112422243324E0E2EA9592F0001FA6
:102C5600111F221F331F001C111C221C331C0416BB
:102C660015062606370688F3041A150A260A370AB1
:102C7600ECCF001F111F221F331F402D512D622D37
:0C2C8600732D0095109520953095089551
:102C9200C895702D3196C895602D3196C895502DE6
:102CA2003196C895402D3196C8953196102C01FA6F
:102CB200C8953196202CC8953196302C0895F1DFB5
:102CC200041B10E003C0EADF041B150B20E030E018
:102CD20005C0DEDF041B150B260B370BC8F010FCFA
:102CE2001AC03AD0402D38D00417100588F446F4A3
:102CF200E00FF11FC895E22DF32DE019F040099481
:102D0200000F111FE00FF11F27D0202C25D0302CEF
:102D1200E22DF32D099411F4BEF7ECCF31960EF0AB
:102D2200319650E060E070E017D0402D4B3F68F0E4
:102D320079F34F3F41F04E3F21F00ED0702D0CD071
:102D4200602D0AD0502D08D0402D041B150B260BE8
:0E2D5200370B11F3E8F2E2CFC89531960895E1
:102D6000BF93AF93A02FB12F02C001900D9241509D
:0A2D70005040D8F7AF91BF910895CD
:102D7A00BF93AF93A02FB12F03C0C89531960D9280
:0C2D8A0041505040D0F7AF91BF91089528
:0E2D9600002401C0019201501040E0F70895A2
:022DA40000002D
:102DA600FA92EA92DA92CA92BA92AA929A928A927D
:102DB6007A926A925A924A92BA93AA939A938A9369
:022DC60008956E
:102DC800FF84EE84DD84CC84BB84AA8499848884BF
:102DD8007F806E805D804C80BB81AA8199818881CB
:0E2DE800F0E00FB6F894CE0FDF1F0FBE089577
:102DF60028813981622F632B79F0E02FF12F6081D2
:102E0600E42FF52F7081671739F40F5F1F4F4F5F5F
:102E16005F4F21503040EECF232B51F0E02FF12FA2
:102E260000811127E42FF52F2081021B104002C0DC
:082E36000027112722960895E0
:102E3E0068817981202F312F062E172E6150704018
:102E4E00012859F0E42FF52F0080E22FF32F019285
:0E2E5E002E2F3F2F4F5F5F4FEFCF229608952C
:102E6C009A938A938A819B81E02FF12F282F392FF7
:102E7C000197232B11F04193F9CF899199912296C7
:022E8C000895A7
:102E8E00E02FF12F3081341739F021910E2F1F2FA3
:0A2E9E002223B1F700271127089541
:102EA800E02FF12F2081222311F03196FBCFE01B78
:082EB800F10B0E2F1F2F0895EE
:00000001FF
